 nullws

 Timestamp is 4be8c309 (Tue May 11 11:38:01 2010)

 Preferred load address is 10000000

 Start         Length     Name                   Class
 0001:00000000 00000004H .CRT$XCA                CODE
 0001:00000004 00000004H .CRT$XCZ                CODE
 0001:00000008 00000004H .CRT$XIA                CODE
 0001:0000000c 00000004H .CRT$XIZ                CODE
 0001:00000010 00000004H .CRT$XPA                CODE
 0001:00000014 00000004H .CRT$XPZ                CODE
 0001:00000018 00000004H .CRT$XTA                CODE
 0001:0000001c 00000004H .CRT$XTZ                CODE
 0001:00000020 0000032cH .rdata                  CODE
 0001:0000034c 00000023H .rdata$debug            CODE
 0001:00000370 00001a74H .text                   CODE
 0001:00001de4 00000018H .xdata                  CODE
 0001:00001dfc 00000028H .idata$2                CODE
 0001:00001e24 00000014H .idata$3                CODE
 0001:00001e38 000000b0H .idata$4                CODE
 0001:00001ee8 000001d4H .idata$6                CODE
 0001:000020c0 00000064H .edata                  CODE
 0002:00000000 000000b0H .idata$5                DATA
 0002:000000b0 00000068H .data                   DATA
 0002:00000118 00000034H .bss                    DATA
 0003:00000000 00000130H .pdata                  DATA

  Address         Publics by Value              Rva+Base       Lib:Object

 0000:00000000       ___safe_se_handler_count   00000000     <absolute>
 0000:00000000       ___safe_se_handler_table   00000000     <absolute>
 0001:00000000       __xc_a                     10001000     corelib0:crt0init.obj
 0001:00000004       __xc_z                     10001004     corelib0:crt0init.obj
 0001:00000008       __xi_a                     10001008     corelib0:crt0init.obj
 0001:0000000c       __xi_z                     1000100c     corelib0:crt0init.obj
 0001:00000010       __xp_a                     10001010     corelib0:crt0init.obj
 0001:00000014       __xp_z                     10001014     corelib0:crt0init.obj
 0001:00000018       __xt_a                     10001018     corelib0:crt0init.obj
 0001:0000001c       __xt_z                     1000101c     corelib0:crt0init.obj
 0001:00000884       WSEGL_GetFunctionTablePointer 10001884 f   null_pvr2d_flip.obj
 0001:00000890       PVR2DGetFrameBuffer        10001890 f   libpvr2d:pvr2dmode.obj
 0001:000008cc       PVR2DGetDeviceInfo         100018cc f   libpvr2d:pvr2dmode.obj
 0001:00000994       PVR2DEnumerateDevices      10001994 f   libpvr2d:pvr2dinit.obj
 0001:00000d64       PVR2DCreateDeviceContext   10001d64 f   libpvr2d:pvr2dinit.obj
 0001:00000f8c       PVR2DDestroyDeviceContext  10001f8c f   libpvr2d:pvr2dinit.obj
 0001:00001090       DestroyFlipChain           10002090 f   libpvr2d:pvr2dflip.obj
 0001:00001160       PVR2DDestroyFlipChain      10002160 f   libpvr2d:pvr2dflip.obj
 0001:000011fc       PVR2DGetFlipChainBuffers   100021fc f   libpvr2d:pvr2dflip.obj
 0001:00001270       PVR2DPresentFlip           10002270 f   libpvr2d:pvr2dflip.obj
 0001:00001310       PVR2DSetPresentFlipProperties 10002310 f   libpvr2d:pvr2dflip.obj
 0001:00001428       PVR2DCreateFlipChain       10002428 f   libpvr2d:pvr2dflip.obj
 0001:000016cc       PVR2DQueryBlitsComplete    100026cc f   libpvr2d:pvr2dblt.obj
 0001:000017a8       DllMain                    100027a8 f   corelib0:dllmain.obj
 0001:000018c4       _DllMainCRTStartup         100028c4 f   corelib0:pegdmain.obj
 0001:000018f4       __GSHandlerCheckCommon     100028f4 f   corelib0:gshandler.obj
 0001:00001930       __GSHandlerCheck           10002930 f   corelib0:gshandler.obj
 0001:00001954       __security_init_cookie     10002954 f   corelib0:seccinit.obj
 0001:000019b0       __security_check_cookie    100029b0 f   corelib0:armsecgs.obj
 0001:000019c4       __gsfailure                100029c4 f   corelib0:armsecgs.obj
 0001:00001ad0       _cexit                     10002ad0 f   corelib0:cexit.obj
 0001:00001aec       _initterm                  10002aec f   corelib0:crt0dat.obj
 0001:00001b20       _cinit                     10002b20 f   corelib0:crt0dat.obj
 0001:00001b54       free                       10002b54 f   corelib1:COREDLL.dll
 0001:00001b64       malloc                     10002b64 f   corelib1:COREDLL.dll
 0001:00001b74       _XcptFilter                10002b74 f   corelib1:COREDLL.dll
 0001:00001b84       __C_specific_handler       10002b84 f   corelib1:COREDLL.dll
 0001:00001b94       __security_gen_cookie2     10002b94 f   corelib1:COREDLL.dll
 0001:00001ba4       __report_gsfailure         10002ba4 f   corelib1:COREDLL.dll
 0001:00001bb4       PVRSRVDisconnect           10002bb4 f   srvclum:SRVCLUM.dll
 0001:00001bc4       PVRSRVCloseDCDevice        10002bc4 f   srvclum:SRVCLUM.dll
 0001:00001bd4       PVRSRVMemCopy              10002bd4 f   srvclum:SRVCLUM.dll
 0001:00001be4       PVRSRVGetDCInfo            10002be4 f   srvclum:SRVCLUM.dll
 0001:00001bf4       PVRSRVOpenDCDevice         10002bf4 f   srvclum:SRVCLUM.dll
 0001:00001c04       PVRSRVFreeUserModeMem      10002c04 f   srvclum:SRVCLUM.dll
 0001:00001c14       PVRSRVCallocUserModeMem    10002c14 f   srvclum:SRVCLUM.dll
 0001:00001c24       PVRSRVAcquireDeviceData    10002c24 f   srvclum:SRVCLUM.dll
 0001:00001c34       PVRSRVEnumerateDevices     10002c34 f   srvclum:SRVCLUM.dll
 0001:00001c44       PVRSRVEnumerateDeviceClass 10002c44 f   srvclum:SRVCLUM.dll
 0001:00001c54       PVRSRVConnect              10002c54 f   srvclum:SRVCLUM.dll
 0001:00001c64       PVRSRVUnmapDeviceClassMemory 10002c64 f   srvclum:SRVCLUM.dll
 0001:00001c74       PVRSRVMapDeviceClassMemory 10002c74 f   srvclum:SRVCLUM.dll
 0001:00001c84       PVRSRVGetDCSystemBuffer    10002c84 f   srvclum:SRVCLUM.dll
 0001:00001c94       PVRSRVEnumDCDims           10002c94 f   srvclum:SRVCLUM.dll
 0001:00001ca4       PVRSRVAllocUserModeMem     10002ca4 f   srvclum:SRVCLUM.dll
 0001:00001cb4       PVRSRVEnumDCFormats        10002cb4 f   srvclum:SRVCLUM.dll
 0001:00001cc4       PVRSRVDestroyDeviceMemContext 10002cc4 f   srvclum:SRVCLUM.dll
 0001:00001cd4       PVRSRVReleaseMiscInfo      10002cd4 f   srvclum:SRVCLUM.dll
 0001:00001ce4       SGXDestroyTransferContext  10002ce4 f   srvclum:SRVCLUM.dll
 0001:00001cf4       SGXCreateTransferContext   10002cf4 f   srvclum:SRVCLUM.dll
 0001:00001d04       PVRSRVCreateDeviceMemContext 10002d04 f   srvclum:SRVCLUM.dll
 0001:00001d14       PVRSRVGetMiscInfo          10002d14 f   srvclum:SRVCLUM.dll
 0001:00001d24       PVRSRVDestroyDCSwapChain   10002d24 f   srvclum:SRVCLUM.dll
 0001:00001d34       PVRSRVSwapToDCSystem       10002d34 f   srvclum:SRVCLUM.dll
 0001:00001d44       PVRSRVSwapToDCBuffer       10002d44 f   srvclum:SRVCLUM.dll
 0001:00001d54       PVRSRVReallocUserModeMem   10002d54 f   srvclum:SRVCLUM.dll
 0001:00001d64       PVRSRVSetDCDstRect         10002d64 f   srvclum:SRVCLUM.dll
 0001:00001d74       PVRSRVGetDCBuffers         10002d74 f   srvclum:SRVCLUM.dll
 0001:00001d84       PVRSRVCreateDCSwapChain    10002d84 f   srvclum:SRVCLUM.dll
 0001:00001d94       PVRSRVEventObjectWait      10002d94 f   srvclum:SRVCLUM.dll
 0001:00001da4       SGX2DQueryBlitsComplete    10002da4 f   srvclum:SRVCLUM.dll
 0001:00001db4       PVRSRVClockus              10002db4 f   srvclum:SRVCLUM.dll
 0001:00001dc4       DisableThreadLibraryCalls  10002dc4 f   coredll:COREDLL.dll
 0001:00001dd4       TerminateProcess           10002dd4 f   coredll:COREDLL.dll
 0001:00001dfc       __IMPORT_DESCRIPTOR_COREDLL 10002dfc     corelib1:COREDLL.dll
 0001:00001e10       __IMPORT_DESCRIPTOR_SRVCLUM 10002e10     srvclum:SRVCLUM.dll
 0001:00001e24       __NULL_IMPORT_DESCRIPTOR   10002e24     corelib1:COREDLL.dll
 0002:00000000       __imp_free                 10004000     corelib1:COREDLL.dll
 0002:00000004       __imp_malloc               10004004     corelib1:COREDLL.dll
 0002:00000008       __imp___rt_udiv            10004008     corelib1:COREDLL.dll
 0002:0000000c       __imp__XcptFilter          1000400c     corelib1:COREDLL.dll
 0002:00000010       __imp___C_specific_handler 10004010     corelib1:COREDLL.dll
 0002:00000014       __imp___security_gen_cookie2 10004014     corelib1:COREDLL.dll
 0002:00000018       __imp___report_gsfailure   10004018     corelib1:COREDLL.dll
 0002:0000001c       __imp_DisableThreadLibraryCalls 1000401c     coredll:COREDLL.dll
 0002:00000020       __imp_TerminateProcess     10004020     coredll:COREDLL.dll
 0002:00000024       \177COREDLL_NULL_THUNK_DATA 10004024     corelib1:COREDLL.dll
 0002:00000028       __imp_PVRSRVMemCopy        10004028     srvclum:SRVCLUM.dll
 0002:0000002c       __imp_PVRSRVGetDCInfo      1000402c     srvclum:SRVCLUM.dll
 0002:00000030       __imp_PVRSRVOpenDCDevice   10004030     srvclum:SRVCLUM.dll
 0002:00000034       __imp_PVRSRVFreeUserModeMem 10004034     srvclum:SRVCLUM.dll
 0002:00000038       __imp_PVRSRVCallocUserModeMem 10004038     srvclum:SRVCLUM.dll
 0002:0000003c       __imp_PVRSRVAcquireDeviceData 1000403c     srvclum:SRVCLUM.dll
 0002:00000040       __imp_PVRSRVEnumerateDevices 10004040     srvclum:SRVCLUM.dll
 0002:00000044       __imp_PVRSRVEnumerateDeviceClass 10004044     srvclum:SRVCLUM.dll
 0002:00000048       __imp_PVRSRVConnect        10004048     srvclum:SRVCLUM.dll
 0002:0000004c       __imp_PVRSRVUnmapDeviceClassMemory 1000404c     srvclum:SRVCLUM.dll
 0002:00000050       __imp_PVRSRVMapDeviceClassMemory 10004050     srvclum:SRVCLUM.dll
 0002:00000054       __imp_PVRSRVGetDCSystemBuffer 10004054     srvclum:SRVCLUM.dll
 0002:00000058       __imp_PVRSRVCloseDCDevice  10004058     srvclum:SRVCLUM.dll
 0002:0000005c       __imp_PVRSRVAllocUserModeMem 1000405c     srvclum:SRVCLUM.dll
 0002:00000060       __imp_PVRSRVEnumDCFormats  10004060     srvclum:SRVCLUM.dll
 0002:00000064       __imp_PVRSRVDestroyDeviceMemContext 10004064     srvclum:SRVCLUM.dll
 0002:00000068       __imp_PVRSRVReleaseMiscInfo 10004068     srvclum:SRVCLUM.dll
 0002:0000006c       __imp_SGXDestroyTransferContext 1000406c     srvclum:SRVCLUM.dll
 0002:00000070       __imp_SGXCreateTransferContext 10004070     srvclum:SRVCLUM.dll
 0002:00000074       __imp_PVRSRVCreateDeviceMemContext 10004074     srvclum:SRVCLUM.dll
 0002:00000078       __imp_PVRSRVGetMiscInfo    10004078     srvclum:SRVCLUM.dll
 0002:0000007c       __imp_PVRSRVDestroyDCSwapChain 1000407c     srvclum:SRVCLUM.dll
 0002:00000080       __imp_PVRSRVSwapToDCSystem 10004080     srvclum:SRVCLUM.dll
 0002:00000084       __imp_PVRSRVSwapToDCBuffer 10004084     srvclum:SRVCLUM.dll
 0002:00000088       __imp_PVRSRVReallocUserModeMem 10004088     srvclum:SRVCLUM.dll
 0002:0000008c       __imp_PVRSRVSetDCDstRect   1000408c     srvclum:SRVCLUM.dll
 0002:00000090       __imp_PVRSRVGetDCBuffers   10004090     srvclum:SRVCLUM.dll
 0002:00000094       __imp_PVRSRVCreateDCSwapChain 10004094     srvclum:SRVCLUM.dll
 0002:00000098       __imp_PVRSRVEventObjectWait 10004098     srvclum:SRVCLUM.dll
 0002:0000009c       __imp_SGX2DQueryBlitsComplete 1000409c     srvclum:SRVCLUM.dll
 0002:000000a0       __imp_PVRSRVClockus        100040a0     srvclum:SRVCLUM.dll
 0002:000000a4       __imp_PVRSRVDisconnect     100040a4     srvclum:SRVCLUM.dll
 0002:000000a8       __imp_PVRSRVEnumDCDims     100040a8     srvclum:SRVCLUM.dll
 0002:000000ac       \177SRVCLUM_NULL_THUNK_DATA 100040ac     srvclum:SRVCLUM.dll
 0002:00000110       __security_cookie          10004110     corelib0:seccinit.obj
 0002:00000114       __security_cookie_complement 10004114     corelib0:seccinit.obj
 0002:0000013c       _exitflag                  1000413c     corelib0:cexit.obj
 0002:00000140       __onexitend                10004140     <common>
 0002:00000144       __onexitbegin              10004144     <common>
 0002:00000148       _pRawDllMain               10004148     <common>

 entry point at        0001:000018c4

 Static symbols

 0001:00000370       WSEGL_IsDisplayValid       10001370 f   null_pvr2d_flip.obj
 0001:00000380       WSEGL_InitialiseDisplay    10001380 f   null_pvr2d_flip.obj
 0001:00000524       WSEGL_CloseDisplay         10001524 f   null_pvr2d_flip.obj
 0001:00000544       WSEGL_CreateWindowDrawable 10001544 f   null_pvr2d_flip.obj
 0001:000006c4       WSEGL_CreatePixmapDrawable 100016c4 f   null_pvr2d_flip.obj
 0001:000006cc       WSEGL_DeleteDrawable       100016cc f   null_pvr2d_flip.obj
 0001:000006f8       WSEGL_SwapDrawable         100016f8 f   null_pvr2d_flip.obj
 0001:00000750       WSEGL_SwapControlInterval  10001750 f   null_pvr2d_flip.obj
 0001:0000079c       WSEGL_WaitNative           1000179c f   null_pvr2d_flip.obj
 0001:000007ac       WSEGL_CopyFromDrawable     100017ac f   null_pvr2d_flip.obj
 0001:000007b4       WSEGL_CopyFromPBuffer      100017b4 f   null_pvr2d_flip.obj
 0001:000007bc       WSEGL_GetDrawableParameters 100017bc f   null_pvr2d_flip.obj
 0001:00000b7c       InitDisplayDevice          10001b7c f   libpvr2d:pvr2dinit.obj
 0001:000017c8       _DllMainCRTStartupHelper   100027c8 f   corelib0:pegdmain.obj
 0001:00001a08       doexit                     10002a08 f   corelib0:cexit.obj
